:020000040800F2
:1000000000040020A1020008990F00089D0F0008BD
:10001000F10F00089D0F0008C50F0008A30200089B
:10002000A3020008A3020008A30200089D330008F1
:10003000A3020008A3020008A3020008A30200080C
:10004000A3020008A3020008A3020008A3020008FC
:10005000A3020008A30200089D370008C937000862
:10006000F5370008213800084D380008A3020008C1
:10007000A3020008A3020008A3020008A3020008CC
:10008000A3020008A3020008A3020008A3020008BC
:10009000A3020008A3020008A302000879380008A0
:1000A000A3020008A3020008A3020008A30200089C
:1000B000A3020008A3020008A3020008A30200088C
:1000C000A3020008A3020008A3020008A30200087C
:1000D000A3020008A3020008A3020008A30200086C
:1000E000E1380008A3020008A3020008A3020008E8
:1000F000A3020008A3020008A3020008A30200084C
:10010000A3020008A302000819340008A302000893
:10011000A3020008A3020008A3020008A30200082B
:10012000A3020008A3020008A3020008A30200081B
:10013000A3020008A3020008A3020008A30200080B
:10014000A3020008A3020008A3020008A3020008FB
:10015000A3020008A3020008A3020008A3020008EB
:10016000A3020008A3020008A3020008A3020008DB
:10017000A3020008E92C0008A3020008A30200085B
:10018000A3020008A3020008913A0008A302000895
:10019000A3020008A3020008A3020008A3020008AB
:1001A000A3020008A3020008A3020008A30200089B
:1001B000A3020008A3020008A3020008A30200088B
:1001C000A3020008A3020008A3020008A30200087B
:1001D000A3020008D52C0008A3020008A30200080F
:1001E000A3020008A3020008A3020008A30200085B
:1001F000A3020008A3020008A3020008A30200084B
:10020000A3020008A3020008A3020008A30200083A
:10021000A3020008A3020008A3020008A30200082A
:10022000A3020008A3020008A3020008A30200081A
:10023000A3020008A3020008A3020008A30200080A
:10024000A3020008A3020008A3020008A3020008FA
:10025000A3020008A3020008A3020008A3020008EA
:10026000A3020008A3020008A3020008A3020008DA
:10027000A3020008A3020008A3020008A3020008CA
:10028000A3020008A3020008A3020008A3020008BA
:10029000A3020008A3020008A3020008A3020008AA
:1002A00002E000F000F8FEE772B6394880F30888F3
:1002B000384880F3098838484EF60851CEF20001DC
:1002C000086040F20000CCF200004EF63471CEF22D
:1002D00000010860BFF34F8FBFF36F8F40F2000043
:1002E000C0F2F0004EF68851CEF200010860BFF374
:1002F0004F8FBFF36F8F4FF00000E1EE100A4EF604
:100300003C71CEF200010860062080F31488BFF330
:100310006F8F01F08BFF02F0BFFF4FF055301F4988
:100320001B4A91423CBF41F8040BFAE71C49194AA9
:1003300091423CBF41F8040BFAE71A491A4A1B4B99
:100340009A423EBF51F8040B42F8040BF8E7002034
:100350001749184A91423CBF41F8040BFAE701F0F3
:10036000A9FF03F00DF8144C144DAC4203DA54F815
:10037000041B8847F9E700F03FF8114C114DAC42DF
:1003800003DA54F8041B8847F9E701F091BF000035
:1003900000040020002400200000000800000020CD
:1003A00000040020304200080024002044240020E3
:1003B000482400205C350020A0020008A0020008AC
:1003C000A0020008A00200082DE9F04F2DED108AD0
:1003D000C1F80CD0D0F80CD0BDEC108ABDE8F08F7D
:1003E000002383F311882846A047002001F078FB02
:1003F00001F028FB00DFFEE738B51F4C6FF07403F7
:10040000002523701C236570A570E570257165714A
:10041000A571E57125726572A372E57200F022FD87
:1004200020B10E2325726572A372E57201F0C0FE41
:10043000044601F0F5FE0546D0B9104B9C4219D098
:1004400001339C4241F2883412BF05460024012545
:10045000002001F0B7FE0DB100F0B6F800F068FD25
:1004600000F058FC204600F06FF900F0ADF8F9E715
:100470000024EDE70446EBE748240020010007B024
:1004800008B500F0E9FBA0F120035842584108BD2F
:10049000054B07B51B88022101A8ADF8043000F018
:1004A00029FC03B05DF804FBF43E0008064991F80E
:1004B000243033B100230822086A81F8243000F088
:1004C0004DBC0120704700BF682400202DE9F84F83
:1004D000234C05468846174694F824308BBB2E469D
:1004E000DFF87C90002F38D094F824A0BAF1000FE8
:1004F00005D12022FF214846266200F007FDCAF1FF
:100500000805414604EB8A00BD4228BF3D465FFA1C
:1005100085FBAD00A7EB0B072A462E4400F0CEFC6E
:1005200094F82430A844FFB29B445FFA8BFBBBF1E4
:10053000080F84F824B0D5D1FFF7B8FF0028D1D137
:1005400008E0266A06EB8306B042C9D0FFF7AEFF8B
:100550000028C4D10020BDE8F88F0120BDE8F88F45
:100560006824002010B5202383F311881248C36843
:100570000BB101F03BFB0023104A4FF47A710E4897
:1005800001F0F8FA002383F311880D4C236813B1AE
:100590002368013B2360636813B16368013B6360B8
:1005A000084B1B7833B9636823B9022000F084FC40
:1005B0003223636010BD00BF54240020650500088D
:1005C0009825002090240020554B56492DE9F041F4
:1005D00053F8042F013201D1BDE8F0818B42F7D1ED
:1005E000514C524B22689A4240F29880504B9B6883
:1005F00003F1006303F500339A4280F08F800020FE
:1006000000F0A4FB02204B4B187000F053FC4A4B47
:10061000D3F8E8200022C3F8E820D3F81011C3F87B
:100620001021D3F81011D3F8EC10C3F8EC20D3F854
:100630001411C3F81421D3F81411D3F8F010C3F82F
:10064000F020D3F81811C3F81821D3F81811D3F8F3
:10065000801041F00061C3F88010D3F8801021F0C1
:100660000061C3F88010D3F88010D3F8801041F0F7
:100670000071C3F88010D3F8801021F00071C3F826
:100680008010D3F8803072B62C4B2D490B601D685A
:100690002468BFF34F8FBFF36F8F2A4BC3F88420BA
:1006A000BFF34F8F5A6922F480325A61BFF34F8FE4
:1006B000D3F8802043F6E07EC2F3C906C2F34E327F
:1006C000B707520102EA0E0838463146013948EAB6
:1006D000000C00F14040B1F1FF3FC3F874C2F5D106
:1006E000203A12F1200FEDD1BFF34F8FBFF36F8F80
:1006F000BFF34F8FBFF36F8F5A6922F400325A61F4
:100700000022C3F85022BFF34F8FBFF36F8F202317
:1007100083F31188AD4685F308882047BDE8F08152
:10072000FCFF01081C00020804000208FFFF01088A
:1007300048240020902400200044025800000208B1
:1007400008ED00E000ED00E02DE9F04F99B0B34C6A
:100750002022FF21019010A8A66800F0D7FBB04A24
:10076000A3461378A3B90121AE481170C3602023BA
:1007700083F31188C3680BB101F038FA0023AA4A49
:100780004FF47A71A74801F0F5F9002383F311883B
:10079000019B13B1A54B019A1A600023A44AA349F7
:1007A000019F99461C461D46984613704B60029265
:1007B000012000F07FFB002F00F012829B4B1B6892
:1007C000002B40F00D8219B0BDE8F08F0220FFF73A
:1007D00057FE002840F0FB81019BB9F1000F08BFD4
:1007E0001F46944B1B8802210BA8ADF82C3000F05B
:1007F00081FADDE74FF47A7000F02EFA031E0393BE
:10080000EADB0220FFF73CFE82460028E4D0039B8F
:10081000581E042800F2DD81DFE800F0030E1114F9
:10082000170018A80523042140F8343D00F062FAAF
:1008300054464FF0000856E004217848F6E70421BA
:100840007D48F3E704217D48F0E71C24204604346A
:1008500000F07EFA04210B900BA800F04BFA2C2C30
:10086000F4D1E5E7002DB7D0002CB5D00220FFF77A
:1008700007FE0546002800F0AF8101206C4C00F017
:1008800065FA4FF000090220207000F013FB5FFAB8
:1008900089FA504600F06AFA074658B1504609F105
:1008A000010900F073FA0028F1D12C46A94600276F
:1008B000634B97E701233E460220237000F0F8FACD
:1008C000DBF808309E4206D2304600F041FA013093
:1008D000EBD10436F4E70026029BA9462C461E7095
:1008E0003746524B5E6000F019FB15B1002C18BF63
:1008F0000027FFF7CDFD5BE7002D3FF46DAF002C27
:100900003FF46AAF0220029B187000F0D3FA322045
:1009100000F0A2F9B0F1000AC0F25E811AF00305FE
:1009200040F05A8106EB0A03DBF80820934200F2FC
:100930005381BAF5807F00F24F8155450DDA4FF4AF
:100940007A7000F089F90490049B002BC0F2448176
:10095000049B3C4AAB540135EFE7C820FFF790FDFC
:100960000546002800F038811F2E11D8C6F120045A
:1009700010AB26F0030033495445184428BF5446B1
:10098000224600F09BFA2246FF212E4800F0BEFAD4
:100990004FEAAA0A2B4930465FFA8AF2FFF796FD22
:1009A0000446002800F01A8106EB8A0605469AE7FD
:1009B0000220FFF765FD00283FF40EAFFFF776FD3C
:1009C00000283FF409AF4FF0000A5346DBF8082037
:1009D00092451CD2BAF11F0F12D8109A01320FD0D3
:1009E0002AF0030218A90A4452F8202C0B92184648
:1009F00004220BA90AF1040A00F00EFB0346E5E706
:100A00005046039300F0A4F9039B0B90EFE718A85E
:100A1000042140F84C3D00F06DF964E748240020C3
:100A20009425002054240020650500089825002006
:100A300090240020F63E00084C2400205024002082
:100A4000F83E00089424002018A80023642140F8F0
:100A5000343D00F02BF900287FF4BEAE0220FFF7F2
:100A60000FFD00283FF4B8AE0B9800F0A1F918ABC9
:100A700043F8480D04211846CDE718A80023642147
:100A800040F8343D00F012F900287FF4A5AE0220B2
:100A9000FFF7F6FC00283FF49FAE0B9800F08AF9B0
:100AA00018AB43F8440DE5E70220FFF7E9FC002806
:100AB0003FF492AE00F084F918AB43F8400DD9E74B
:100AC0000220FFF7DDFC00283FF486AE0BA91420BE
:100AD00000F07CF9824618A8042140F83CAD00F0F3
:100AE00009F951460BA896E7322000F0B5F8B0F1AD
:100AF000000AFFF671AE1AF0030F7FF46DAE0AEB39
:100B00000803DBF8082093423FF666AE0220FFF7A9
:100B1000B7FC00283FF460AE2AF0030AC244D04577
:100B20003FF4E1AE404608F1040800F011F9042159
:100B30000A900AA800F0DEF8F1E74FF47A70FFF7A8
:100B40009FFC00283FF448AEFFF7B0FC00283FF4BC
:100B5000AFAE109B01330CD0082210A90020FFF784
:100B6000B5FC00283FF4A4AE2022FF2110A800F01D
:100B7000CDF9FFF78DFC374800F0B8FF23E6002DD4
:100B80003FF42AAE002C3FF427AE18A800236421BE
:100B900040F8343D00F08AF8824600287FF41CAE0D
:100BA0000220FFF76DFC00283FF416AE0390FFF71C
:100BB0006FFC41F28830574600F098FF0B9800F028
:100BC000E9F900F0ABF9039B1C461D46F0E505462C
:100BD00089E64FF00008FFE52546FDE52C4667E66F
:100BE000002000F039F80490049B002BFFF6E3ADE1
:100BF000012000F05DF9049B213B122B3FF6D8AD9C
:100C000001A252F823F000BFCD070008F507000845
:100C100065080008B1070008B1070008B10700081F
:100C2000F9080008E90A0008B1090008490A0008A3
:100C30007B0A0008A90A0008B1070008C10A0008D9
:100C4000B10700083B0B0008E7080008B1070008DF
:100C50007F0B0008A0860100114B37B51A780024DD
:100C6000014601328DF80740D2B2012A11D80D4851
:100C7000012203681D6A4FF47A734B430DF107019B
:100C8000A847012805D1084B9DF807001C7003B048
:100C900030BD4FF4FA7000F029FF4FF0FF30F6E757
:100CA0000024002080260020BC25002038B50E4BF3
:100CB00005461A780132D2B2012A0ED80B48042216
:100CC00003681C6A4FF47A734B432946A0470428F3
:100CD00003D10020064B187038BD4FF4FA7000F0B5
:100CE00005FF4FF0FF3038BD002400208026002093
:100CF000BC25002030B4054C0A4601462368204636
:100D0000DD69034BAC4630BC604700BF8026002045
:100D1000A0860100F8B50A4C00250A4E01F030F912
:100D2000094F207030682378834207D901F024F9F5
:100D3000336805440133BD423360F3D9F8BD00BFC9
:100D4000BD250020A0250020FFFF010001F0E4B92F
:100D500000F1006000F500300068704700F10060AD
:100D6000920000F5003001F067B90000054B1A68E9
:100D7000054B1B789B1A834202D9104401F0FCB842
:100D800000207047A0250020BD25002038B5074D64
:100D900004462868204401F0F5F828B92868204462
:100DA000BDE8384001F000B938BD00BFA0250020E3
:100DB00000207047014BC058704700BF00E8F11F8A
:100DC000014B1868704700BF0010005C234BF0B562
:100DD000234C1B682788C3F30B0665681B0C94F92A
:100DE0000820BE4228D0A789BE4206D101220C2588
:100DF00005FB0244656894F9082041F20104A3420E
:100E00001CD041F20304A3421AD042F20104A342CF
:100E100018D042F20304A34208BF5622441E013DEB
:100E20000B460C44A34217D215F9016F581C5EB152
:100E3000034600F8016CF5E70022D8E75A22EDE7F7
:100E40005922EBE75822E9E72C2584421D7001D98D
:100E5000981C5A70401AF0BD1846FBE70010005C61
:100E600004240020104B41F201015B888B429AB2AE
:100E700011D041F203018B420FD042F201039A429A
:100E80000DD042F203039A420BD10323074A02EB2F
:100E90008303D87870470023F8E70123F6E702239D
:100EA000F4E70020704700BF0010005CFC3E000823
:100EB000704700007047000070470000002310B525
:100EC000934203D0CC5CC4540133F9E710BD000059
:100ED00030B5441E14F9010F0B4658B193F9005078
:100EE0000131854206D11AB993F90020801A30BD2C
:100EF000013AEFE7002AF7D1104630BD024603461B
:100F0000981A13F9011B0029FAD1704702440346CD
:100F1000934202D003F8011BFAE77047024B1A789C
:100F2000024B1A70704700BFBC250020002400202F
:100F300038B5134D134C284600F00AF921462846CF
:100F400000F032F924681048D4F89020D2F8043820
:100F500043F00203C2F8043800F0C8FD0B492046F4
:100F600000F032FAD4F89020D2F8043823F00203CB
:100F7000C2F804384FF4E132054B1A6038BD00BFA7
:100F800080260020A43F000840420F00CC3F00080C
:100F9000A425002070470000FEE7000000B59BB0CC
:100FA000EFF3098168226846FFF788FFEFF30583B6
:100FB000034B9A6B9A6A9A6A9A6A9A6A9B6AFEE7E4
:100FC00000ED00E000B59BB0EFF3098168226846B0
:100FD000FFF774FFEFF30583044B9A6B9A6A9A6AE2
:100FE0009A6A9A6A9A6A9B6AFEE700BF00ED00E07F
:100FF00000B59BB0EFF3098168226846FFF75EFFFA
:10100000EFF30583034B5A6B9A6A9A6A9A6A9A6A53
:101010009B6AFEE700ED00E030B50A44074D9142BF
:101020000BD011F8013B09245840013CF7D040F3A4
:1010300000032B4083EA5000F7E730BD2083B8ED72
:10104000002304491A465A50C81808334260802BBE
:10105000F9D17047C0250020026843681143016040
:1010600003B118477047000013B5446BD4F89434AB
:101070001A681178042915D1217C022912D1197915
:10108000012312898B4013420CD101A904F14C00B9
:1010900001F072FFD4F894440246019B2179206844
:1010A00000F0EAF902B010BD143001F0F5BE000006
:1010B0004FF0FF33143001F0EFBE00004C3001F070
:1010C000C7BF00004FF0FF334C3001F0C1BF00003C
:1010D000143001F0C3BE00004FF0FF31143001F0B6
:1010E000BDBE00004C3001F093BF00004FF0FF3256
:1010F0004C3001F08DBF0000D0F8942438B513684F
:1011000005461978042901D0012038BD017C022947
:10111000FAD1127901205C8990400440F4D105F1A4
:10112000140001F055FE02460028EDD0D5F8945485
:101130004FF480732868697900F08CF9204638BD37
:10114000406BFFF7D9BF00000020704770470000D8
:101150007FB5124B01250226044603600023057467
:1011600000F18402436029468360C3600C4B029007
:10117000143001934FF48073009601F005FE094B83
:1011800004F523722946019304F14C004FF4807357
:101190000294009601F0CCFE04B070BD283F000818
:1011A00041110008691000080A68202383F31188A0
:1011B0000B790B3342F823004B79133342F82300A9
:1011C0008B7913B10B3342F823000223C0F8941437
:1011D0000374002383F311887047000038B5037F40
:1011E000044613B190F85430ABB90125201D0221FB
:1011F000FFF732FF04F1140025776FF0010100F0D2
:101200009DFC84F8545004F14C006FF00101BDE8DE
:10121000384000F093BC38BD10B5012104460430BD
:10122000FFF71AFF0023237784F8543010BD000025
:1012300038B504460025143001F0BEFD04F14C0021
:10124000257701F08DFE201D84F854500121FFF711
:1012500003FF2046BDE83840FFF74EBF90F88030CE
:1012600003F06003202B19D190F88120212A0AD0A5
:10127000222A4FF000030ED0202A0FD1084A4267DD
:101280000722826704E0064B436707238367002336
:10129000C3670120704743678367F9E70020704701
:1012A0001C240020D0F8943437B51A68044611780D
:1012B00004291AD1017C022917D119790123128935
:1012C0008B40134211D100F14C05284601F008FF74
:1012D00058B101A9284601F04FFED4F894440246C3
:1012E000019B2179206800F0C7F803B030BD0000F1
:1012F00001F10B03F7B550F8234005460E46F4B153
:10130000202383F3118805EB8607201D08214C3428
:10131000FFF7A2FEFB685B691B6813B1204601F072
:1013200039FE01A9204601F027FE024648B1019B83
:101330003146284600F0A0F8002383F3118803B05B
:10134000F0BDFB685A691268002AF5D01B8A013B80
:101350001340F1D105F18002EAE70000133138B5FE
:1013600050F82140DCB1202383F31188D4F8942471
:101370001368527903EB8203DB689B695D6845B1B2
:1013800004216018FFF768FE294604F1140001F0FB
:1013900029FD2046FFF7B0FE002383F3118838BDF6
:1013A0007047000001F00EB8012300F1300200F197
:1013B000500103700023436042F8043B8A42D3612A
:1013C000FAD103814381704738B50446202383F363
:1013D0001188002500F10C0300F13002416043F850
:1013E000045B9342FBD1204601F00EF802232370E8
:1013F00085F3118838BD000070B500EB8103054608
:1014000050690E461446DA6018B110220021FFF729
:101410007DFDA06918B110220021FFF777FD31464C
:101420002846BDE8704001F001B90000038900F1D1
:101430003002002103F001030381438903F001031B
:10144000438100F1100343F8041B9342FBD101F0E8
:1014500085B90000F0B4012500EB810447898D4077
:10146000E4683D43A469458123600023A260636072
:10147000F0BC01F0A1B90000F0B4012500EB81043B
:1014800007898D40E4683D4364690581236000233A
:10149000A2606360F0BC01F019BA0000022300F101
:1014A0000C0200F1300110B5037004460023A0F8CF
:1014B000883080F88A3080F88B300381438142F88D
:1014C000043B8A42FBD184F87030204601F042F898
:1014D00063681B6823B120460021BDE8104018470F
:1014E00010BD00000278436880F88C2005221B683C
:1014F00002700BB10421184770470000436890F850
:101500008C201B6802700BB1052118477047000042
:1015100090F8703070B5044613B1002380F8703035
:1015200004F18002204601F03DF963689B6863BBCB
:1015300094F8805015F0600615D194F8813005F0CC
:101540007F0545EA032540F202339D4200F00E81FB
:101550005BD8022D00F0DC803FD8002D00F08780A2
:10156000012D00F0CF800021204601F0D3FB0021A7
:10157000204601F0C3FB63681B6813B106212046B7
:101580009847062384F8703070BD2046984700289D
:10159000CED094F8872094F8863043EA0223A26FD5
:1015A000934238BFA36794F98030A56F002B4FF0AA
:1015B000200380F2FD80002D00F0EC80092284F8E9
:1015C000702083F311880021A36F626F2046FFF71C
:1015D00053FF002383F3118870BDB5F5817F00F0C0
:1015E000B180B5F5407F49D0B5F5807FBBD194F887
:1015F0008230012BB7D1B4F8883023F00203A4F86D
:1016000088306667A667E667C3E740F201639D42DC
:101610001ED8B5F5C06F3BD2B5F5A06FA3D1B4F815
:101620008030B3F5A06F0ED194F88230204684F854
:101630008A3000F0EDFF63681B6813B1012120467A
:1016400098470323237000236367A367E367A0E73A
:10165000B5F5106F32D040F602439D4252D0B5F539
:10166000006F80D104F18B036367012324E004F150
:101670008803E56763670223A3678AE794F88230EB
:10168000012B7FF470AFB4F8883043F00203B6E763
:1016900094F885202046616894F884304D6843EAC8
:1016A000022394F8831094F88220A84700283FF47E
:1016B0005AAF436863670368A367A4E72378042BE2
:1016C00010D1202383F311882046FFF7AFFE86F365
:1016D00011886368032184F88B601B6821700BB14B
:1016E0002046984794F88230002BACD084F88B3099
:1016F0000423237063681B68002BA4D002212046BA
:101700009847A0E7374B63670223A36700239DE751
:1017100094F88410204611F0800F01F00F010ED0D4
:1017200001F032F8012806D002287FF41CAF2E4BBE
:10173000A067636767E72D4BA567636763E701F001
:1017400015F8EFE794F88230002B7FF40CAF94F893
:10175000843013F00F013FF476AF1A06204602D50D
:1017600001F0F0FA6FE701F0E1FA6CE794F88230EB
:10177000002B7FF4F8AE94F8843013F00F013FF49F
:1017800062AF1B06204602D501F0C4FA5BE701F008
:10179000B5FA58E7142284F8702083F311882B4699
:1017A0002A4629462046FFF755FE85F3118870BD6D
:1017B0005DB1152284F8702083F311880021A36F96
:1017C000626F2046FFF746FE03E70B2284F8702085
:1017D00083F311882B462A4629462046FFF74CFE04
:1017E000E3E700BF583F0008503F0008543F00089F
:1017F00038B590F870300446152B29D8DFE803F08F
:101800003E28282828283E28280B29392828282837
:10181000282828283E3E90F8871090F88620836F6D
:1018200042EA01229A4214D9C268128AB3FBF2F545
:1018300002FB15356DB9202383F311882B462A4608
:101840002946FFF719FE85F311880A2384F87030C2
:1018500038BD142384F87030202383F311880023CB
:1018600020461A461946FFF7F5FD002383F3118839
:1018700038BDC36F03B198470023E7E7002101F0AB
:1018800049FA0021204601F039FA63681B6813B158
:101890000621204698470623D8E7000090F87020DC
:1018A000152A38B5044622D80123934040F64162F8
:1018B00013421DD113F480150FD19B0217D50B23B2
:1018C00080F87030202383F311882B462A4629465E
:1018D000FFF7D2FD85F3118838BDC3689B695B684B
:1018E0002BB9C36F03B19847002384F8703038BD1B
:1018F000002101F00FFA0021204601F0FFF9636892
:101900001B6813B10621204698470623EDE7000027
:10191000024B00221B605B609A60704740260020EB
:10192000002382680374054B1B6899689142FBD2BF
:101930005A6803604260106058607047402600207B
:1019400008B5202383F31188037C032B05D0042BD7
:101950000DD02BB983F3118808BD436900221A60AA
:101960004FF0FF334361FFF7DBFF0023F2E790E81E
:101970000C001A6002685360F2E7000000238268DE
:101980000374054B1B6899689142FBD85A68036041
:10199000426010605860704740260020054B19696E
:1019A00008741868026853601A6018610123037490
:1019B000FEF70ABD402600204B1C30B5054687B017
:1019C0000A4C10D0236901A8094A00F0D3F8284630
:1019D000FFF7E4FF049B13B101A800F007F92369A6
:1019E000586907B030BDFFF7D9FFF8E7402600205F
:1019F0004119000838B50C4D044641612B698168D6
:101A00009A68914203D8BDE83840FFF789BF18466D
:101A1000FFF786FF01232C61014623742046BDE8B1
:101A20003840FEF7D1BC00BF40260020044B1A68A6
:101A30001B6990689B68984294BF00200120704702
:101A40004026002010B5084C236820691A685460AD
:101A50002260012223611A74FFF790FF014620697A
:101A6000BDE81040FEF7B0BC402600208260022294
:101A700002740022427470478368A3F17C0243F829
:101A80000C2C026943F83C2C426943F8382C074A75
:101A900043F81C2CC268A3F1180043F8102C022252
:101AA00003F8082C002203F8072C7047E103000814
:101AB00010B5202383F31188FFF7DEFF00210446D1
:101AC000FFF798FF002383F31188204610BD000024
:101AD000024B1B6958610F20FFF760BF40260020B2
:101AE000202383F31188FFF7F3BF000008B50146F8
:101AF000202383F311880820FFF75EFF002383F380
:101B0000118808BD49B1064B42681B6918605A60CC
:101B1000136043600420FFF74FBF4FF0FF30704762
:101B2000402600200368984206D01A680260506080
:101B300018465961FFF7F4BE7047000038B50446F7
:101B40000D462068844200D138BD036823605C6084
:101B50004561FFF7E5FEF4E7054B03F114025A6116
:101B60009A614FF0FF32DA6100221A62704700BFBB
:101B700040260020F8B5036102291A4B0646C260D0
:101B800038BF02215C6A184B1A461F4652F8145F90
:101B900095420AD1586198611C6205604560816078
:101BA0000819BDE8F84001F0BDBA186AAB68241AFC
:101BB0000C1902D3E41A2D6804E09C4202D220449E
:101BC00001F0C0FAAB689C42F4D86B683560736072
:101BD0001E604FF0FF336E60B460A968091BA960F6
:101BE000FB61F8BD000C00404026002010B41A4CE8
:101BF000234653F8141F814210D0416802680A60DE
:101C0000026851609A424FF00001C16003D09368AE
:101C100081680B4493605DF8044B70470A680020AC
:101C20009A4262615360C86003D15DF8044B01F0D1
:101C300083BA936888680344206A9360074A526AAB
:101C4000121A9342E7D9991A5DF8044B012998BFFB
:101C5000931C184401F076BA40260020000C004086
:101C600000207047FEE70000704700004FF0FF3093
:101C700070470000022906D0032906D00129064832
:101C800018BF0020704705487047032A9ABF0448D0
:101C900000EBC2000020704728400008DC3F00082D
:101CA0002424002070B59AB006460846144601ADBB
:101CB000294600F095F82846FFF720F9C0B2431CEA
:101CC0005B0086E8180023700323023404F8013C0B
:101CD00000231946DAB20234904201D81AB070BD1E
:101CE000EA5C013304F8011C04F8022CF2E700005E
:101CF00008B5202383F311880348FFF7D3FA0023A4
:101D000083F3118808BD00BF8026002010B504466B
:101D1000052916D8DFE801F016150316161D202335
:101D200083F311880E4A0121FFF766FB20460D4A16
:101D30000221FFF761FB0C48FFF77AFA002383F3D7
:101D4000118810BD202383F311880748FFF746FA56
:101D5000F4E7202383F311880348FFF75DFAEDE7EA
:101D60005C3F0008803F00088026002038B50C4DFD
:101D70000C4C2A460C4904F10800FFF793FF05F1CB
:101D8000CA0204F110000949FFF78CFF05F5CA7279
:101D900004F118000649BDE83840FFF783BF00BFD3
:101DA000482B002024240020AC3F0008B63F000848
:101DB000C13F000870B5044608460D46FFF79EF87F
:101DC000C6B22046013403780BB9184670BD3246BE
:101DD0002946FFF77DF80028F3D1012070BD0000EF
:101DE0002DE9F84F05460C46FFF788F82C49C6B296
:101DF0002846FFF7DFFF08B10336F6B22949284627
:101E0000FFF7D8FF08B11036F6B2632E0DD8DFF811
:101E10009080DFF89090244FDFF894A0DFF894B022
:101E20002E7846B92670BDE8F88F29462046BDE8D1
:101E3000F84F02F057B8252E2ED1072241462846EA
:101E4000FFF746F870B9DBF8003007350A3444F87C
:101E50000A3CDBF8043044F8063CBBF8083024F8B0
:101E6000023CDDE7082249462846FFF731F898B9D9
:101E7000A21C0E4B13F8011F023209095345C95D1C
:101E800002F8041C197801F00F01C95D02F8031C67
:101E9000F0D118340835C3E7267001350134BFE7A7
:101EA00048400008C13F00085B400008FFE7F11F01
:101EB0000BE8F11F50400008BFF34F8F044B1A6925
:101EC0005107FCD1D3F810215207F8D1704700BF59
:101ED0000020005208B50D4B1B78ABB9FFF7ECFFA3
:101EE0000B4BDA68D10704D50A4A5A6002F18832EE
:101EF0005A60D3F80C21D20706D5064AC3F804214C
:101F000002F18832C3F8042108BD00BFA62D0020CD
:101F1000002000522301674508B5114B1B78F3B927
:101F2000104B1A69510703D5DA6842F04002DA60B3
:101F3000D3F81021520705D5D3F80C2142F0400206
:101F4000C3F80C21FFF7B8FF064BDA6842F0010234
:101F5000DA60D3F80C2142F00102C3F80C2108BD6D
:101F6000A62D0020002000520E289ABF00F58060A8
:101F700040040020704700004FF40030704700001C
:101F80000F2070470E2808B50BD8FFF7EDFF00F5BE
:101F900000330268013204D104308342F9D10120B8
:101FA00008BD002008BD00000E2810B504463FD82B
:101FB000FFF782FFFFF78EFF1E484FF0FF33072C1D
:101FC0004361C0F814311DD80361FFF775FF230288
:101FD00043F02403C360C36843F08003C360036914
:101FE0005A07FCD4FFF768FF2046FFF7BDFF4FF408
:101FF000003100F0F7F8FFF78FFF2046BDE81040F2
:10200000FFF7C0BFC0F81031FFF756FFA4F1080377
:102010001B0243F02403C0F80C31D0F80C3143F01C
:102020008003C0F80C31D0F810315B07FBD4D9E73E
:10203000002010BD002000522DE9F84F40EA0203B5
:1020400005460E461746DB0656D13446DFF8C090EB
:10205000DFF8C0A0FFF73EFF3B1B33441F2B04D823
:10206000FFF75AFF0120BDE8F88F202221462846BD
:1020700001F028FF002837D005F17843214A224893
:102080009342224B98BF984603F5827392BFD34682
:10209000C8469B46A3F1080388BF1846FFF70CFF0C
:1020A0004FF0FF3304F11C01A5EB040ECBF8003018
:1020B000036843F002030360231FD8F8002012F0E6
:1020C000050FFAD153F8042F99424EF80320F4D1AA
:1020D000BFF34F8FFFF7F0FE4FF0FF33CBF8003028
:1020E000036823F00203036020222146284601F002
:1020F000E9FE20B1FFF710FF0020BDE8F88F203582
:102100002034A9E7FFFF0F000C20005210200052DE
:10211000102100521420005210B5084C237828B129
:1021200053B9FFF7D7FE0123237010BD23B12070F0
:10213000BDE81040FFF7F0BE10BD00BFA62D002087
:1021400002440439064BD2B210B5904200D110BD02
:10215000441C00B253F8200041F8040FE0B2F4E749
:10216000504000580F4B30B51C6F240405D41C6F31
:102170001C671C6F44F400441C670B4C0244043978
:102180002368D2B243F480732360084B904200D19D
:1021900030BD441C51F8045F00B243F82050E0B257
:1021A000F4E700BF0044025800480258504000586D
:1021B00007B5012201A90020FFF7C2FF019803B073
:1021C0005DF804FB13B50446FFF7F2FFA04206D00A
:1021D00002A90122002041F8044DFFF7C3FF02B01D
:1021E00010BD00000144BFF34F8F064B884204D35B
:1021F000BFF34F8FBFF36F8F7047C3F85C0220307F
:10220000F4E700BF00ED00E0034B1B685B0142BF39
:102210000122024B1A707047D0440258A72D0020AB
:10222000014B1878704700BFA72D0020F0B5BFF311
:102230004F8FBFF36F8F1D4B0021C3F85012BFF3B8
:102240004F8FBFF36F8F5A6942F400325A61BFF368
:102250004F8FBFF36F8FC3F88410BFF34F8FD3F846
:10226000802043F6E076C2F3C904C2F34E32A507DC
:10227000520102EA060E284621464EEA00070139BD
:1022800000F14040C3F860724F1CF6D1203A12F1C1
:10229000200FEED1BFF34F8F5A6942F480325A615A
:1022A000BFF34F8FBFF36F8FF0BD00BF00ED00E0B5
:1022B000FEE70000084A094B09498B4204D3094A4A
:1022C0000021934205D3704752F8040F43F8040BE2
:1022D000F3E743F8041BF4E7704200085C35002084
:1022E0005C3500205C350020D0F89430002230B5F9
:1022F0001146D0F890409D684FF0FF3004EB421338
:1023000001329542C3F80019C3F81019C3F808093F
:10231000C3F8001BC3F8101BC3F8080BEED24FF034
:102320000113C4F81C3830BD00EB81032DE9F04FD8
:10233000D3F80CE04F1C4FEA4118DEF814403F037D
:10234000D4F800C06568D0F8902065450AD3012014
:10235000D2F8343800FA01F123EA0101C2F8341846
:10236000BDE8F08FACEB0503BEF81060B34228BFA8
:10237000334602EB0806D6F81869B6B2B3EB860FFF
:1023800013D8A6683A449946A6F1040A5AF804BF3D
:10239000B9F1040FC2F800B002D9A9F10409F5E7B8
:1023A0001E442B44A6606360CCE70020BDE8F08F9C
:1023B000890141F02001016103699B06FCD41220D0
:1023C00000F050BF10B50A4C2046FEF7EDFF094B58
:1023D000C4F89030084BC4F89430084C2046FEF7FF
:1023E000E3FF074BC4F89030064BC4F8943010BD9F
:1023F000A82D00200000084090400008442E002036
:10240000000004409C4000080378012B70B505468D
:102410005DD1494BD0F89040984259D1474B0E219D
:102420006520D3F8D82042F00062C3F8D820D3F852
:10243000002142F00062C3F80021D3F80021D3F854
:10244000802042F00062C3F88020D3F8802022F080
:102450000062C3F88020D3F8803000F07FFC384B56
:10246000E360384BC4F800380023D5F89060C4F816
:10247000003EC02323604FF40413A3633369002B91
:10248000FCDA01230C20336100F0ECFE3369DB073A
:10249000FCD4122000F0E6FE3369002BFCDA0026A3
:1024A0002846A660FFF720FF6B68C4F81068DB6859
:1024B000C4F81468C4F81C68002B3AD1224BA361FD
:1024C0004FF0FF336361A36843F00103A36070BD65
:1024D0001E4B9842C8D1194B0E214D20D3F8D8205D
:1024E00042F00072C3F8D820D3F8002142F0007205
:1024F000C3F80021D3F80021D3F8802042F0007205
:10250000C3F88020D3F8802022F00072C3F8802026
:10251000D3F88020D3F8D82022F08062C3F8D820E6
:10252000D3F8002122F08062C3F80021D3F80031F3
:1025300093E7074BC3E700BFA82D002000440258D3
:102540004014004003002002003C30C0442E002014
:10255000083C30C0F8B5D0F89040054600214FF057
:1025600000662046FFF724FFD5F8941000234FF0B3
:1025700001128F684FF0FF30C4F83438C4F81C28BB
:1025800004EB431201339F42C2F80069C2F8006BAA
:10259000C2F80809C2F8080BF2D20B68D5F89020EF
:1025A000C5F89830636210231361166916F010069F
:1025B000FBD1122000F056FED4F8003823F4FE635D
:1025C000C4F80038A36943F4402343F01003A36127
:1025D0000923C4F81038C4F814380B4BEB604FF0E3
:1025E000C043C4F8103B094BC4F8003BC4F8106961
:1025F000C4F80039D5F8983003F1100243F4801381
:10260000C5F89820A362F8BD6C4000084080001017
:10261000D0F8902090F88A10D2F8003823F4FE63A6
:1026200043EA0113C2F80038704700002DE9F04179
:102630000EB20D4600EB8608D8F80C100F6807F0B4
:102640000303022B53D0032B53D03F4A3F4F012BA0
:1026500018BF1746D0F890404FEA451E002205F1FA
:10266000100C04EB0E03C3F8102B8A69002A42D029
:102670004A8A05F158033A435B01E2500123D4F83A
:102680001C2803FA0CF31343C4F81C38A644002397
:102690004A69CEF8103905F13F03002A3BD00A8A77
:1026A00004EB8303898B9208012988BF4A43D0F841
:1026B0009810561841EA02422946C0F89860204610
:1026C0005A60FFF775FED8F80C301B8A43EA855331
:1026D0001F4305F148035B01E7500123D4F81C2890
:1026E00003FA05F51543C4F81C58BDE8F081184FEE
:1026F000B0E7184FAEE704EB4613D3F8002B22F4F3
:102700000042C3F8002B0123D4F81C2803FA0CF371
:1027100022EA0303B8E704EB83030F4A04EB4616EF
:1027200029465A602046FFF743FED6F800390122B9
:1027300023F4004302FA05F5C6F80039D4F81C3832
:1027400023EA0505CFE700BF0080001000800410D9
:102750000080081000800C1000040002D0F89420C3
:102760001268C0F89820FFF7BFBD00005831D0F8BC
:10277000903049015B5813F4004004D013F4001F5B
:1027800014BF0120022070474831D0F89030490131
:102790005B5813F4004004D013F4001F14BF012051
:1027A0000220704700EB8101CB68196A0B68136047
:1027B0004B6853607047000000EB810330B5DD6863
:1027C000AA691368D36019B9402B84BF40231360F2
:1027D0006B8A1468D0F890201C4402EB4110013C35
:1027E00009B2B4FBF3F46343033323F0030343EA76
:1027F000C44343F0C043C0F8103B2B6803F003030D
:10280000012B0ED1D2F8083802EB411013F4807F6F
:10281000D0F8003B14BF43F0805343F00053C0F89E
:10282000003B02EB4112D2F8003B43F00443C2F8F4
:10283000003B30BD2DE9F041D0F8906005460C46D4
:1028400006EB4113D3F8087B3A07C3F8087B08D599
:10285000D6F814381B0704D500EB8103DB685B68EE
:102860009847FA072FD5D6F81438DB072BD505EB98
:102870008403D968CCB98B69488A5E68B6FBF0F2EC
:1028800000FB12628AB91868DA6890420DD2121AF7
:1028900083E81400202383F3118821462846FFF79C
:1028A0008BFF84F31188BDE8F081012303FA04F261
:1028B0006B8923EA02036B81CB6823B1214628464A
:1028C000BDE8F0411847BDE8F081000000EB81034E
:1028D0004A0170B5DD68D0F890306C692668E66012
:1028E00056BB1A444FF40020C2F810092A6802F0BF
:1028F0000302012A0AB20ED1D3F8080803EB4214EE
:1029000010F4807FD4F8000914BF40F0805040F0EC
:102910000050C4F8000903EB4212D2F8000940F05D
:102920000440C2F800090122D3F8340802FA01F188
:102930000143C3F8341870BD19B9402E84BF40203C
:10294000206020681A442E8A841940F00050013C0F
:10295000B4FBF6F440EAC440C6E700002DE9F041BC
:10296000D0F8906004460D4606EB4113D3F8087981
:10297000C3F80879FB071CD5D6F81038DA0718D544
:1029800000EB8103D3F80CE0DEF81430D3F800C07C
:10299000DA6894451BD2A2EB0C024FF000081A60D3
:1029A000C3F80480202383F31188FFF78FFF88F397
:1029B00011883B0618D50123D6F83428AB401342C2
:1029C00012D029462046BDE8F041FFF7ADBC0123F7
:1029D00003FA01F2038923EA02030381DEF80830D7
:1029E000002BE6D09847E4E7BDE8F0812DE9F047F9
:1029F000D0F8905004466E69AB691E40F1046E61D8
:102A000003D5BDE8F047FEF749BD002E12DAD5F830
:102A1000003E9A0705D0D5F8003E23F00303C5F821
:102A2000003ED5F80438204623F00103C5F80438E9
:102A3000FEF764FD330502D52046FEF753FDB704CB
:102A40000CD5D5F8083813F0060FEB6823F4705353
:102A50000CBF43F4105343F4A053EB60300704D58C
:102A60006368DB680BB120469847F10200F1A18052
:102A7000B2020BD5D4F8908000274FF00109D4F8AA
:102A80009430F9B29B688B4280F0D280F3061AD55D
:102A9000D4F890100A6AC2F30A1702F00F0302F486
:102AA000F012B2F5802F00F0EB80B2F5402F0AD182
:102AB00004EB830301F58051DB68186A00231A4692
:102AC0009F4240F0D1803003D5F8185835D5E9033E
:102AD00003D500212046FFF7ADFEAA0303D501214F
:102AE0002046FFF7A7FE6B0303D502212046FFF720
:102AF000A1FE2F0303D503212046FFF79BFEE8022A
:102B000003D504212046FFF795FEA90203D5052130
:102B10002046FFF78FFE6A0203D506212046FFF705
:102B200089FE2B0203D507212046FFF783FEEF0124
:102B300003D508212046FFF77DFE700340F1C780D2
:102B4000E90703D500212046FFF708FFAA0703D5B0
:102B500001212046FFF702FF6B0703D50221204623
:102B6000FFF7FCFE2F0703D503212046FFF7F6FEF3
:102B7000EE0603D504212046FFF7F0FEA80603D594
:102B800005212046FFF7EAFE690603D50621204607
:102B9000FFF7E4FE2A0603D507212046FFF7DEFEF5
:102BA000EB0540F1948020460821BDE8F047FFF78F
:102BB000D5BED4F890904FF000084FF0010AD4F839
:102BC00094305FFA88F79B68BB42FFF451AF09EB82
:102BD0004713D3F8002902F44022B2F5802F24D104
:102BE000D3F80029002A20DAD3F8002942F09042D5
:102BF000C3F80029D3F80029002AFBDB3946D4F8B2
:102C00009000FFF7D5FB22890AFA07F322EA0303B3
:102C1000238104EB8703DB689B6813B139462046A8
:102C2000984739462046FFF77FFB08F10108C6E7C1
:102C300008EB4112D2F8003B03F44023B3F5802F98
:102C400010D1D2F8003B002B0CDA628909FA01F3AB
:102C500022EA0303638104EB8103DB68DB680BB1C9
:102C60002046984701370AE713F0030F00D10A689E
:102C7000072B03F101039EBF0270120A01301FE708
:102C800004EB830301F58051DA6890690268D0F89B
:102C900008C04068A2EB000E00221046974208D1FF
:102CA000DB689B699A683A449A605A6817445F6087
:102CB00009E712F0030F00D10868964502F10102FE
:102CC00082BF8CF80000000A0CF1010CE6E7BDE8B9
:102CD000F087000008B50348FFF788FEBDE808400C
:102CE00000F06CBBA82D002008B50348FFF77EFE5E
:102CF000BDE8084000F062BB442E0020D0F89030C0
:102D000003EB4111D1F8003B43F40013C1F8003B41
:102D100070470000D0F8903003EB4111D1F8003932
:102D200043F40013C1F8003970470000D0F8903028
:102D300003EB4111D1F8003B23F40013C1F8003B31
:102D400070470000D0F8903003EB4111D1F8003902
:102D500023F40013C1F800397047000000F160430C
:102D600000F01F020901400903F56143C9B2800068
:102D700083F80013012300F16040934000F56140A7
:102D8000C0F880310360704730B50433039C017292
:102D9000002104FB0325C361049B00600363059BC2
:102DA0004060C16042610261856104624262816289
:102DB000C162436330BD00000022416AC2604161CC
:102DC00001616FF001018262C262FEF7B7BE0000CE
:102DD00003694269934203D1C2680AB10020704777
:102DE000181D7047036919600021C2680132C26072
:102DF000C269134482699342036124BF436A036139
:102E0000FEF790BE38B504460D46E3683BB16269F3
:102E10000020131D1268A3621344E36238BD237AB5
:102E200033B929462046FEF76DFE0028EDDA38BD9D
:102E30006FF00100FBE70000C368C269013BC3609B
:102E40004369134482699342436124BF436A4361E7
:102E500000238362036B03B11847704770B52023CA
:102E6000044683F31188866A3EB9FFF7CBFF054617
:102E700018B186F31188284670BDA36AE26A13F878
:102E8000015B9342A36202D32046FFF7D5FF0023E4
:102E900083F31188EFE700002DE9F84F04460E4652
:102EA00090469946202787F311880025AA46D4F832
:102EB00028B0BBF1000F09D149462046FFF7A2FF19
:102EC00020B18BF311882846BDE8F88FA16AA8EBE2
:102ED000050BE36A5B1A9B4528BF9B46BBF1400F7D
:102EE0001BD9334601F1400251F8040B914243F8DB
:102EF000040BF9D1A36A403640354033A362A26A7D
:102F0000E36A9A4202D32046FFF796FF8AF31188BC
:102F10004545D8D287F31188C9E730465A46FDF7B0
:102F2000CDFFA36A5E445D445B44A362E7E7000013
:102F300010B5029C04330172C36103FB042100231A
:102F400000608362C362039B40600363049BC460B0
:102F500042610261816104624262436310BD00000C
:102F6000026A6FF00101C260426A4261026100229E
:102F70008262C262FEF7E2BD436902699A4203D1EE
:102F8000C2680AB100207047184650F8043B0B6035
:102F900070470000C3680021C2690133C360436900
:102FA000134482699342436124BF436A4361FEF73D
:102FB000B9BD000038B504460D46E3683BB123694E
:102FC00000201A1DA262E2691344E36238BD237A2D
:102FD00033B929462046FEF795FD0028EDDA38BDC5
:102FE0006FF00100FBE7000003691960C268013A55
:102FF000C260C269134482699342036124BF436A79
:10300000036100238362036B03B11847704700001C
:1030100070B5202304460E4683F31188856A35B9BE
:103020001146FFF7C7FF10B185F3118870BDA36A81
:103030001E70A36AE26A01339342A36204D3E1697A
:1030400020460439FFF7D0FF002080F3118870BDBF
:103050002DE9F84F04460D4691469A464FF0200858
:1030600088F311880026B346A76A4FB95146204617
:10307000FFF7A0FF20B187F311883046BDE8F88F35
:10308000A06AA9EB0603E76A3F1A9F4228BF1F46C2
:10309000402F1BD905F1400355F8042B9D4240F801
:1030A000042BF9D1A36A40364033A362A26AE36AD3
:1030B0009A4204D3E16920460439FFF795FF8BF368
:1030C00011884E45D9D288F31188CDE729463A4672
:1030D000FDF7F4FEA36A3D443E443B44A362E5E7AA
:1030E000026943699A4203D1C3681BB91846704705
:1030F0000023FBE7836A002BF8D0043B9B1AF5D032
:103100001360C368013BC360C3691A4483699A4270
:10311000026124BF436A0361002383620123E5E760
:1031200000F08EB9034B002258631A610222DA6064
:10313000704700BF000C00400022014BDA6070476E
:10314000000C0040014B5863704700BF000C00406A
:10315000FEE7000010B5194CFEF7DAFBFEF7FCFCA9
:10316000802217492046FEF781FC012344F8180C01
:103170000374144B144AD96821F4E0610904090C62
:103180000A431249DA60CA6842F08072CA60104A83
:103190001049C2F8B01F116841F0010111601022FE
:1031A000DA77202283F82220002383F3118862B685
:1031B0000948BDE81040FEF77BBC00BF6826002030
:1031C000A840000800ED00E00003FA05F0ED00E083
:1031D000001000E055CEACC5B04000082DE9F84F16
:1031E0001E4C4FF00008DFF87890656904F1140771
:1031F000D9F82430266AAA689E1B96421CD34FF049
:10320000200AAA68236AD5F80CB0B61A13442362C0
:103210002B68BB425F606361C5F80C8001D1FFF78A
:103220008BFF88F311882869D8478AF3118865696C
:10323000AB689E42E5D2DBE76269BA420CD0916886
:1032400023628E1B9660A86802282CBF1818981C51
:10325000BDE8F84FFFF776BFBDE8F88F40260020A5
:10326000000C0040034B59685A68521A9042FBD830
:10327000704700BF001000E04B6843608B688360BC
:10328000CB68C3600B6943614B6903628B6943621E
:103290000B6803607047000008B52C4B40F2FF71CB
:1032A0002B48D3F888200A43C3F88820D3F8882015
:1032B00022F4FF6222F00702C3F88820D3F88820A6
:1032C000D3F8E0200A43C3F8E020D3F808210A43EA
:1032D000C3F808211F4AD3F808311146FFF7CCFF85
:1032E0001D4802F11C01FFF7C7FF1C4802F138011D
:1032F000FFF7C2FF1A4802F15401FFF7BDFF19485A
:1033000002F17001FFF7B8FF174802F18C01FFF7D7
:10331000B3FF164802F1A801FFF7AEFF144802F10F
:10332000C401FFF7A9FF134802F1E001FFF7A4FF72
:10333000114802F1FC01FFF79FFF104802F58C7164
:10334000FFF79AFFBDE8084000F054B90044025866
:1033500000000258D040000800040258000802583B
:10336000000C0258001002580014025800180258AD
:10337000001C02580020025800240258002802585D
:1033800008B500F007FBFFF7E5FEFEF73DFFBDE8DF
:103390000840FEF7EBBC000070470000064A536887
:1033A00023F001035360EFF30983683383F3098843
:1033B000002383F31188704730EF00E010B520231D
:1033C00083F31188104B5B6813F4006318D0F1EE9F
:1033D000103AEFF309844FF0807344F84C3C0B4BE8
:1033E000DB6844F8083CA4F1680383F30988FEF71E
:1033F0001DFB18B1064B44F8503C10BD054BFAE7D5
:1034000083F3118810BD00BF00ED00E030EF00E055
:10341000F1030008F4030008084B1A69920710B57D
:1034200008D500241C61202383F31188FFF7D6FE02
:1034300084F31188BDE81040FFF7C0BF000C0040C6
:10344000124B08213220D3F8E82042F00802C3F8DA
:10345000E820D3F8102142F00802C3F810210C4AEA
:10346000D3F81031D36B43F00803D363C722094B61
:103470009A624FF0FF32DA6200229A615A63DA6090
:103480005A6001225A611A60FFF768BC0044025872
:103490000010005C000C0040F8B5514B0024D3F83C
:1034A00080204FF0FF32C3F88020D3F88010C3F89B
:1034B0008040D3F88010D3F88410C3F88420D3F868
:1034C0008410C3F88440D3F88410D96F41F0FF41D1
:1034D00041F4FF0141F4DF4141F07F01D967D96F29
:1034E00021F0FF4121F4FF0121F4DF4121F07F01B0
:1034F000D967D96FD3F888106FEA41516FEA5151FB
:10350000C3F88810D3F88810C1F30A01C3F88810F3
:10351000D3F88810D3F89010C3F89020D3F8901007
:10352000C3F89040D3F89010D3F89410C3F89420C7
:10353000D3F89410C3F89440D3F89410D3F89810AB
:10354000C3F89820D3F89810C3F89840D3F898108F
:10355000D3F88C10C3F88C20D3F88C10C3F88C40AF
:10356000D3F88C10D3F89C10C3F89C20D3F89C207F
:10357000C3F89C40D3F89C3000F0ECF9194B0722BB
:103580009A60194ADA60194A1A6105225A60184A83
:10359000536A43F480335362C2F88440BFF34F8FC1
:1035A000D2F8803043F6E076C3F3C904C3F34E3358
:1035B000A5075B0103EA060E284621464EEA0007EE
:1035C000013900F14040C2F874724F1CF6D1203B23
:1035D00013F1200FEED1BFF34F8FBFF36F8FF8BD04
:1035E0000044025890ED00E0000004301B00080386
:1035F00000ED00E001225B4B5B491A605B4B1960F8
:103600009A605B4ADA6000221A614FF440429A6184
:103610009A699204FCD51A6842F480721A60554B7C
:103620001A6F12F4407F04D04FF480321A670022E0
:103630001A671A6842F001021A604E4A134611686E
:103640004807FCD5002111611A6912F03802FBD13C
:10365000012119604FF0804159605A67464ADA6289
:10366000464A1A611A6842F4A0221A60414A134677
:1036700011688903FCD5116841F0800111601A6856
:10368000D205FCD53E4A3F499A6200225A6319632B
:10369000A1F58021DA634B3999635A643A4A1A6476
:1036A0003A4ADA621A6842F0A8521A60314B1A6834
:1036B00002F02852B2F1285FF9D1482222219A6102
:1036C0004FF48862DA6140221A624FF00052DA64E5
:1036D0001A652F4A5A652F4A9A652F4A11601A694E
:1036E00042F003021A61234B1A6902F03802182AC9
:1036F000FAD1D3F8DC2042F00052C3F8DC20D3F832
:10370000042142F00052C3F80421D3F80421D3F875
:10371000DC2042F08042C3F8DC20D3F8042142F0E0
:103720008042C3F80421D3F80421D3F8DC2042F00E
:103730000042C3F8DC20D3F8042142F00042C3F871
:103740000421D3F80421D3F8F42042F00202C3F894
:10375000F420D3F81C2142F00202C3F81C21D3F854
:103760001C3170470881005100C000F00048025829
:1037700002000001004402580000FF010088900888
:10378000121020006302070147040508FD0BFF012A
:103790000010E0000001010000200052084A08B5B6
:1037A000936811680B4003F00103936023B1054A4D
:1037B00013680BB150689847BDE80840FFF7FEBD9D
:1037C00080000058C0250020084A08B59368116899
:1037D0000B4003F00203936023B1054A93680BB1D9
:1037E000D0689847BDE80840FFF7E8BD8000005862
:1037F000C0250020084A08B5936811680B4003F003
:103800000403936023B1054A13690BB150699847CB
:10381000BDE80840FFF7D2BD80000058C025002059
:10382000084A08B5936811680B4003F008039360D9
:1038300023B1054A93690BB1D0699847BDE80840A8
:10384000FFF7BCBD80000058C0250020084A08B51D
:10385000936811680B4003F01003936023B1054A8D
:10386000136A0BB1506A9847BDE80840FFF7A6BD40
:1038700080000058C0250020174B10B59C681A68BE
:10388000144004F478729A60A30604D5134A936A2C
:103890000BB1D06A9847600604D5104A136B0BB180
:1038A000506B9847210604D50C4A936B0BB1D06B33
:1038B0009847E20504D5094A136C0BB1506C984740
:1038C000A30504D5054A936C0BB1D06C9847BDE8AD
:1038D0001040FFF773BD00BF80000058C0250020D6
:1038E0001A4B10B59C681A68144004F47C429A6024
:1038F000620504D5164A136D0BB1506D9847230528
:1039000004D5134A936D0BB1D06D9847E00404D5EC
:103910000F4A136E0BB1506E9847A10404D50C4AA0
:10392000936E0BB1D06E9847620404D5084A136FAA
:103930000BB1506F9847230404D5054A936F0BB120
:10394000D06F9847BDE81040FFF738BD80000058A1
:10395000C0250020062108B50846FFF7FFF906211B
:103960000720FFF7FBF906210820FFF7F7F90621EA
:103970000920FFF7F3F906210A20FFF7EFF90621E6
:103980001720FFF7EBF906212820BDE80840FFF7D4
:10399000E5B9000008B5FFF77FFDFDF751FB00F02A
:1039A0003DF8FDF7FFFCFDF7D1FBFFF7F5FCBDE8A7
:1039B0000840FFF7B5BB000002684368114301608F
:1039C00003B1184770470000143000F0C9B9000077
:1039D0004FF0FF33143000F0C3B90000383000F06E
:1039E0003FBA00004FF0FF33383000F039BA000022
:1039F000143000F08FB900004FF0FF31143000F0A8
:103A000089B90000383000F0E9B900004FF0FF320A
:103A1000383000F0E3B900000020704700F0C2B871
:103A2000044B0360002343608360C360012303747D
:103A3000704700BF0442000838B5C36904460D460C
:103A40001BB904210844FFF7B7FF294604F114000D
:103A500000F044F9002806DA201D4FF48061BDE82B
:103A60003840FFF7A9BF38BD024A136843F0C003CE
:103A70001360704700780040044B5A6810439A68FE
:103A800058600AB1181D1047704700BFF030002081
:103A90002DE9F84F414EF56D2F68EC6921072C6236
:103AA00019D014F0080F0CBF00208020E20748BF97
:103AB00040F02000A3074FF0200348BF40F0400033
:103AC000610748BF40F4807083F31188FFF7D4FF8B
:103AD000002383F31188E20509D5202383F311889D
:103AE0004FF40070FFF7C8FF002383F311884FF0F5
:103AF0002009DFF8A8A04FF0000B14F0200832D105
:103B00003B0615D54FF02009DFF894A020060FD50D
:103B100089F31188504600F089F9002830DA08202E
:103B2000FFF7AAFF27F080032B60002383F311889F
:103B300079060DD562060BD5202383F31188F26C2C
:103B4000336D9A4201D1336C03BB002383F3118898
:103B5000E30604D5B26E13690BB150699847BDE80E
:103B6000F84FFFF72BBC89F31188AB8C504696F8C1
:103B700064101940FFF760FF8BF31188EC69BCE714
:103B800080B2288588F31188EC69BFE727F04007E9
:103B90001020FFF771FF2F60D7E700BFF030002043
:103BA0002831002013B5104C2046FFF739FF04F1EF
:103BB0001400009400234FF400720C4900F080F8C8
:103BC00004F1380000944FF40072094B094900F0E9
:103BD000F9F8094B0C215220E365084B236602B02B
:103BE000BDE81040FFF7BAB8F03000205C3100208B
:103BF000693A00085C3300200078004000E1F505D8
:103C0000F8B51546826804460B46AA4200D285687C
:103C1000A1692669761AB54207D218462A46FDF7E9
:103C20004DF9A3692B44A3610DE011D9AF1B3246B6
:103C30001846FDF743F93A46E1683044FDF73EF98E
:103C4000E2683A44A261A36828465B1BA360F8BD02
:103C500018462A46FDF732F9E368E4E783689342A1
:103C60002DE9F04104460F46154600D2856860698B
:103C70002669361AB54207D22A463946FDF71EF99B
:103C800063692B4463610EE013D9A5EB0608324645
:103C90003946FDF713F94246B919E068FDF70EF908
:103CA000E26842446261A36828465B1BA360BDE8EA
:103CB000F0812A463946FDF701F9E368E2E70000A2
:103CC00010B50A440024C361029B00604060846018
:103CD000C160816141610261036210BD08B5826902
:103CE0004369934201D1826882B98268013282605D
:103CF0005A1C42611970426903699A4201D3C36830
:103D000043610021FDF70EFF002008BD4FF0FF309A
:103D100008BD000070B5202304460E4683F31188C9
:103D2000A568A5B1A368A269013BA360531CA36168
:103D300015782269934224BFE368A361E3690BB15C
:103D400020469847002383F31188284670BD3146EA
:103D50002046FDF7D7FE0028E2DA85F3118870BD12
:103D60002DE9F74F05460F4690469A46D0F81C902D
:103D7000202686F311884FF0000B144664B12246CA
:103D800039462846FFF73CFF034668B951462846A6
:103D9000FDF7B8FE0028F1D0002383F31188A8EBCB
:103DA000040003B0BDE8F08FB9F1000F03D001901B
:103DB0002846C847019B8BF31188E41A1F4486F3F9
:103DC0001188DBE7C160816141611144C361009BDF
:103DD000006040608260016103627047F8B504468C
:103DE0000E461746202383F31188A568A5B1A36862
:103DF000013BA36063695A1C62611E70236962699A
:103E00009A4224BFE3686361E3690BB12046984797
:103E1000002080F31188F8BD39462046FDF772FE78
:103E20000028E2DA85F31188F8BD00008369426951
:103E30009A4210B501D182687AB9826801328260F3
:103E40005A1C82611C7803699A4201D3C36883615A
:103E50000021FDF767FE204610BD4FF0FF3010BD7A
:103E60002DE9F74F05460F4690469A46D0F81C902C
:103E7000202686F311884FF0000B144664B12246C9
:103E800039462846FFF7EAFE034668B951462846F8
:103E9000FDF738FE0028F1D0002383F31188A8EB4A
:103EA000040003B0BDE8F08FB9F1000F03D001901A
:103EB0002846C847019B8BF31188E41A1F4486F3F8
:103EC0001188DBE710B501390244904201D100208E
:103ED00010BD10F8013B11F8014FA342F5D0181B9B
:103EE00010BD0000034611F8012B03F8012B002A36
:103EF000F9D17047121012131211000001105A006C
:103F000003105900012058000320560053544D332C
:103F10003248373F3F3F0053544D333248373433F4
:103F20002F3735330000000000000000C5100008E6
:103F3000B1100008ED100008D9100008E5100008C5
:103F4000D1100008BD100008A91000084911000890
:103F5000000000000100000000000000020000005E
:103F600000000000F11200085D130008400040004E
:103F7000182B0020282B0020020000000000000069
:103F80000300000000000000A11300080000000072
:103F900010000000382B002000000000010000008D
:103FA00000000000A82D002001010200417264758C
:103FB00050696C6F740025424F415244252D424C8C
:103FC000002553455249414C250000000D1D0008B5
:103FD000751C00085D120008F11C00084300000079
:103FE000E43F000809024300020100C03209040056
:103FF0000001020201000524001001052401000156
:10400000042402020524060001070582030800FFBC
:1040100009040100020A0000000705010240000037
:104020000705810240000000120000003040000837
:104030001201100102000040091241570002010262
:10404000030100000403090425424F4152442500A6
:104050004E75636C656F483734330030313233341A
:1040600035363738394142434445460000000000A8
:1040700011150008F11700089D18000840004000C5
:10408000E02E0020E02E002001000000F02E002095
:104090008000000040010000080000000001000056
:1040A00000040000080000006D61696E000000005F
:1040B000C8400008F82E0020F03000200100000069
:1040C000513100080000000069646C6500000000C8
:1040D0000001802A00000000AAAAAAAA000100008C
:1040E000FFFF00000000000000A00A000000000028
:1040F00000000000AAAAAAAA00000000FFFF00001A
:10410000000000000000000000400000000000006F
:10411000AAAAAAAA00400000FFFF000000000000B9
:10412000000000000000000000000000AAAAAAAAE7
:1041300000000000FFFF0000000000000000000081
:104140000000020000000000AAAAAAAA00000100C4
:10415000FFFF00000000000007000000002000003A
:1041600000000000AAAAAAAA00100000FFFF000099
:104170000000000700000000000000000000000038
:10418000AAAAAAAA00000000FFFF00000000000089
:10419000000000000000000000000000AAAAAAAA77
:1041A00000000000FFFF0000000000000000000011
:1041B0000000000000000000AAAAAAAA0000000057
:1041C000FFFF0000000000000000000000000000F1
:1041D00000000000AAAAAAAA00000000FFFF000039
:1041E00000000000000000000000000000000000CF
:1041F000AAAAAAAA00000000FFFF00000000000019
:104200000000000000000000E5390008D139000876
:104210000D3A0008F9390008053A0008F13900089C
:10422000DD390008C9390008193A0008000000000B
:10423000FF000000000000000C3F00083F000000ED
:1042400050040000173F00083F00000000960000E7
:1042500000000800040000004440000800000000C6
:10426000000000000000000000000000000000004E
:04427000000000004A
:00000001FF
